:040000006CEF00F0B1
:10000800FFFFFACF02F0FBCF03F0E9CF04F0EACF0D
:1000180005F0E1CF06F0E2CF07F0D9CF08F0DACF4C
:1000280009F0F3CF0AF0F4CF0BF0F6CF0CF0F7CFCE
:100038000DF0F8CF0EF0F5CF0FF09DAA01D001D04A
:1000480017D09EAA01D001D013D0C80ECF6EE00EF3
:10005800CE6ECD804E50010D0101000EF324D96EF5
:10006800DA6A0101010EDA22AECFDFFF4E2A00D094
:100078009DA001D001D00ED09EA001D001D00AD001
:100088009D9A9E90CD90016E010E000100019B6F1C
:10009800015000D00FC0F5FF0EC0F8FF0DC0F7FFEC
:1000A8000CC0F6FF0BC0F4FF0AC0F3FF09C0DAFF6B
:1000B80008C0D9FF07C0E2FF06C0E1FF05C0EAFF9C
:1000C80004C0E9FF03C0FBFF02C0FAFF1100FFFFF5
:1000D800F9EF0AF0FFFF61EC0BF064EC09F0000E99
:1000E800856E9484000E00010001856F000E0001EA
:1000F800866F000E0001876F000E0001886F0001F7
:10010800606F000E00010001846F000160513F0E16
:1001180000010001846501D001D002D024D023D091
:100128000001606F010E106E0001605144EC0BF08D
:10013800105000010001852711500001000186239D
:10014800000E000100018723000E00010001882332
:1001580000010001842B3F0E00010001846501D0DD
:1001680001D0DED700D0000185C060F0000186C054
:1001780061F0000187C062F0000188C063F0070EDB
:1001880006D00001D8906333623361336033E82EC0
:10019800F8D760C085F061C086F062C087F063C0A0
:1001A80088F085C093F086C094F087C095F088C029
:1001B80096F09494030E000100019D6FFF0E00015C
:1001C8009C6F000100019D51000100018D6F9CC0D2
:1001D8008EF000D0000E00010001856F000E0001B6
:1001E800866F000E0001876F000E0001886F000106
:1001F800606F000E00010001846F000160513F0E26
:1002080000010001846501D001D002D024D023D0A0
:100218000001606F000E106E0001605144EC0BF09D
:1002280010500001000185271150000100018623AC
:10023800000E000100018723000E00010001882341
:1002480000010001842B3F0E00010001846501D0EC
:1002580001D0DED700D0000185C060F0000186C063
:1002680061F0000187C062F0000188C063F0070EEA
:1002780006D00001D8906333623361336033E82ECF
:10028800F8D760C085F061C086F062C087F063C0AF
:1002980088F0A00E146E5A0E156E320E166E000EF1
:1002A800176E85C010F086C011F087C012F088C0A4
:1002B80013F0C6EC0AF010C01CF011C01DF012C0FB
:1002C8001EF013C01FF0FF0E206E030E216E000EED
:1002D800226E000E236E14EC09F01CC097F01DC0AE
:1002E80098F01EC099F01FC09AF0000E000100019E
:1002F800856F000E0001866F000E0001876F000EEB
:100308000001886F0001606F000E00010001846F1A
:10031800000160513F0E00010001846501D001D049
:1003280002D024D023D00001606F010E106E0001AE
:10033800605144EC0BF0105000010001852711506A
:10034800000100018623000E000100018723000E32
:1003580000010001882300010001842B3F0E0001E9
:100368000001846501D001D0DED700D0000185C02E
:1003780060F0000186C061F0000187C062F00001F2
:1003880088C063F0070E06D00001D890633362334B
:1003980061336033E82EF8D7000160510001000195
:1003A800935D0001615100010001945900016251FF
:1003B800000100019559000163510001000196599F
:1003C800D8B001D001D046D0000193C060F0000140
:1003D80094C061F0000195C062F0000196C063F01E
:1003E8000001601F611F621F631F602B000E6123E5
:1003F80062236323000185C064F0000186C065F0B4
:10040800000187C066F0000188C067F0070E06D0BB
:100418000001D8906733663365336433E82EF8D724
:10042800000160510001642500010001856F000191
:100438006151000165210001866F000162510001D0
:1004480066210001876F00016351000167210001E7
:10045800886F0ED0000E00010001856F000E0001AC
:10046800866F000E0001876F000E0001886F00D0B4
:10047800FF0E206E030E216E000E226E000E236EFC
:10048800A00E146E5A0E156E320E166E000E176EF2
:1004980085C010F086C011F087C012F088C013F034
:1004A800C6EC0AF010C01CF011C01DF012C01EF0FE
:1004B80013C01FF014EC09F01CC07CF01DC07DF0C7
:1004C8001EC07EF01FC07FF07CC01CF07DC01DF0F8
:1004D8007EC01EF07FC01FF0C90E206E000E216E78
:1004E800000E226E000E236E14EC09F01CC08FF073
:1004F8001DC090F01EC091F01FC092F097C01CF074
:1005080098C01DF099C01EF09AC01FF0E80E206E2A
:10051800030E216E000E226E000E236E14EC09F0FD
:100528001DC01CF01EC01DF01FC01EF01F6A1C500D
:1005380000010001896F97C01CF098C01DF099C098
:100548001EF09AC01FF0E80E206E030E216E000EFA
:10055800226E000E236E14EC09F01C5000010001FD
:100568008A6F90C08BF08FC08CF0000100018D5114
:10057800000100019D6F000100018E5100019C6F78
:1005880097C01CF098C01DF099C01EF09AC01FF0CB
:10059800E80E206E030E216E000E226E000E236EF2
:1005A80014EC09F01CC080F01DC081F01EC082F060
:1005B8001FC083F00001000E3A6E0001680E396E0C
:1005C800FF0E3C6ED50E3B6E80C03DF081C03EF004
:1005D80082C03FF083C040F05FEC06F00001000EDF
:1005E800186E0001680E176E0001606F000E196E1C
:1005F800000160510001616F010E1A6E0001615126
:100608000001626F000E1B6E0001625191EC07F051
:100618000001000E3A6E0001680E396EFF0E3C6E46
:10062800C60E3B6E8FC03DF090C03EF091C03FF0CB
:1006380092C040F05FEC06F00001000E186E000159
:10064800680E176E0001606F000E196E0001605190
:100658000001616F020E1A6E000161510001626FA4
:10066800000E1B6E0001625191EC07F08FC014F070
:1006780090C015F091C016F092C017F0E80E206EE9
:10068800030E216E000E226E000E236E97C01CF022
:1006980098C01DF099C01EF09AC01FF014EC09F024
:1006A8001CC010F01DC011F01EC012F01FC013F0C6
:1006B800C6EC0AF010C02AF011C02BF012C02CF0C2
:1006C80013C02DF0E80E2E6E030E2F6E000E306E46
:1006D800000E316E90EC08F02AC080F02BC081F03B
:1006E8002CC082F02DC083F00001000E3A6E00018C
:1006F800680E396EFF0E3C6EE40E3B6E80C03DF016
:1007080081C03EF082C03FF083C040F05FEC06F04D
:100718000001000E186E0001680E176E0001606F70
:10072800000E196E000160510001616F060E1A6E0D
:10073800000161510001626F000E1B6E00016251E1
:1007480091EC07F00001000E3A6E0001680E396E58
:10075800FF0E3C6EF30E3B6E9CC03DF09DC03EF01C
:100768005FEC06F00001000E186E0001680E176EAF
:100778000001606F000E196E000160510001616F89
:10078800040E1A6E000161510001626F000E1B6EAB
:100798000001625191EC07F081B201D001D017D06D
:1007A800000100019D519C11D8B401D001D00FD097
:1007B800000100019C07D8A09D07000100019D5180
:1007C800000100018D6F9CC08EF001D000D081BA6D
:1007D80001D001D019D0FF0E000100019C5D030E6D
:1007E80000019D59D8B001D001D00ED00001000100
:1007F8009C4B9D2B000100019D51000100018D6F54
:100808009CC08EF001D000D000019CC060F00001B7
:100818009DC061F00001D890613360330001D89029
:100828006133603300016051BE6E000100019C51CC
:10083800030B0F09BD6E000100019C29030ED8B4FB
:100848009D19D8A401D001D002D0948402D09494E8
:1008580000D0000100019B05D8A401D001D0BAD472
:100868000001606F000E000100019B6F00016051E4
:1008780049EC04F00001606F000E4E6E00016051FB
:100888009D8AA8D4A7D46CEF00F0FFFF01010101F5
:100898000051550AD8B401D001D002D00AD209D2E9
:1008A8004EC01EF0FE0E1E260101000E1E24D96E3B
:1008B800DA6A0101010EDA22DF501F6E4EC020F005
:1008C800FF0E20260101000E2024D96EDA6A0101EC
:1008D800010EDA22DF50236E1F50226E0101010E35
:1008E800116E0101000E106EFE0E4E24126E136A78
:1008F800FF0E132201EC0AF010C024F011C025F0FD
:100908002550231802E124502218D8B401D001D070
:1009180002D0CFD1CED11E6E550E02010201006F5A
:100928001E50BAD1010101010351010102C11EF09B
:100938001F6A1EC01FF01E6A1E10296E1F502A6EE5
:10094800010101010551010104C11EF01F6A1EC009
:100958001FF01E6A1E10276E1F50286E020E295C9B
:10096800000E2A58D8A001D001D015D001010101EC
:100978000151800902010201016F1E6E020E02017F
:100988000201026F1E501E6E030E196E1E50B3EC4C
:1009980009F08FD18ED129042A10D8A401D001D012
:1009A80009D0020E275C000E2858D8B001D001D01B
:1009B8000AD000D0030E275C000E2858D8A001D01A
:1009C80001D016D000D001010101015180090201B6
:1009D8000201016F1E6E030E02010201026F1E501A
:1009E8001E6E030E196E1E50B3EC09F062D161D170
:1009F80001C101F22750272402010201026F1E6E75
:100A0800000E266E1E5038D0265029241E6E000176
:100A1800890E1E24D96EDA6A0001000EDA2226C079
:100A28001FF0030E1F260201000E1F24E16EE26A6A
:100A38000201020EE222DFCFE7FF265029241E6EB4
:100A4800010E1E260001890E1E24D96EDA6A0001E5
:100A5800000EDA2226C01FF0040E1F260201000E27
:100A68001F24E16EE26A0201020EE222DFCFE7FFF5
:100A78002650020F266E00D0D89027341E6E2834D8
:100A88001F6E2650206E216A1E50205C1F50215870
:100A9800D8A001D001D0B8D700D027502724030F01
:100AA800196EB3EC09F005D104D10101010103511C
:100AB800010102C11EF01F6A1EC01FF01E6A1E102F
:100AC800296E1F502A6E010101010551010104C15F
:100AD8001EF01F6A1EC01FF01E6A1E10276E1F50D0
:100AE800286E2950020A2A10D8B401D001D015D096
:100AF800010101010151800902010201016F1E6E0D
:100B0800020E02010201026F1E501E6E030E196EC4
:100B18001E50B3EC09F0CDD0CCD0020E275C000EED
:100B28002858D8A001D001D015D0010101010151E8
:100B3800800902010201016F1E6E030E020102010B
:100B4800026F1E501E6E030E196E1E50B3EC09F094
:100B5800B0D0AFD001C101F2275027240201020111
:100B6800026F29C01EF0020E1E260001890E1E24E7
:100B7800D96EDA6A0001000EDA22DF5002010201A2
:100B8800036F29C01EF0030E1E260001890E1E24C5
:100B9800D96EDA6A0001000EDA22DF500201020182
:100BA800046F27502724030F196EB3EC09F081D086
:100BB80080D0010101010351010102C11EF01F6A29
:100BC8001EC01FF01E6A1E10296E1F502A6E295063
:100BD800020A2A10D8B401D001D015D001010101B0
:100BE8000151800902010201016F1E6E020E02010D
:100BF8000201026F1E501E6E030E196E1E50B3ECDA
:100C080009F057D056D0010121EE03F0030EDF643E
:100C180001D001D015D00101010101518009020163
:100C28000201016F1E6E030E02010201026F1E50C7
:100C38001E6E030E196E1E50B3EC09F03AD039D06F
:100C480001C101F202C102F203C103F204C104F2BC
:100C580005C105F204C18DF005C18EF01E6E060EA9
:100C6800196E1E50B3EC09F024D023D00101010104
:100C78000151800902010201016F1E6E010E02017D
:100C88000201026F1E501E6E030E196E1E50B3EC49
:100C980009F00FD00ED00DD0010101010151030A56
:100CA800D8B403D7070AD8B43DD6020AD8B481D736
:100CB800DDD71200FFFFFFFF000E466E3D0E456EAA
:100CC8000DD14D50250AD8B401D001D009D039C072
:100CD800D9FF3AC0DAFF4DC0DFFF394A3A2AFED0C1
:100CE800416E000E476E415008D007D00DD147889D
:100CF80004D021D020D0F2D01ED03B50416E3C50C1
:100D0800426E3B4A3C2A41C0F6FF42C0F7FF000E44
:100D1800F86E0800FFFFF5CF4DF04D50000AD8B42B
:100D2800F3D0640AD8B407D00D0AD8B404D0050AA1
:100D3800D8B4DDD7D3D047A801D001D011D045C051
:100D4800D9FF46C0DAFFDECF48F0DECF49F0DECF6C
:100D58004AF0DECF4BF0040E4526000E462212D094
:100D680045C0D9FF46C0DAFFDECF48F0DDCF49F0F5
:100D7800000E49BEFF0E4A6E4B6E020E4526000E4F
:100D8800462200D04BAE01D001D00BD0030E471243
:100D98004B1E4A1E491E486C000E49224A224B220D
:100DA80000D0416E010E4D6E41504D500A0AD8A434
:100DB80001D001D002D02AD029D04D50040D9E0E6A
:100DC800F324F66EF76AFF0EF722F86A000EF8228F
:100DD8000900FFFFF550485C0900FFFFF55049582E
:100DE8000900FFFFF5504A580900FFFFF5504B581E
:100DF800D8B001D001D002D009D008D04D2A4D502A
:100E08000A0AD8A401D001D0D8D700D04750030B84
:100E1800D8B401D001D009D039C0D9FF3AC0DAFF1F
:100E28002D0EDF6E394A3A2A00D04D50436E446A7F
:100E380043BE440647D043C041F0D8904136D890CD
:100E480041369E0E4124F66EF76AFF0EF722F86AC5
:100E5800000EF8220900FFFFF5CF20F00900FFFF80
:100E6800F5CF21F00900FFFFF5CF22F00A00FFFFC0
:100E7800F5CF23F048C01CF049C01DF04AC01EF051
:100E88004BC01FF014EC09F01CC02AF01DC02BF059
:100E98001EC02CF01FC02DF00A0E2E6E000E2F6EF5
:100EA800000E306E000E316E47EC0AF02A50300FFB
:100EB8004D6E39C0D9FF3AC0DAFF4DC0DFFF394A5D
:100EC8003A2A00D04306D8A044064328D8B4442878
:100ED800D8A401D001D0AFD701D000D03B50416E8B
:100EE8003C50426E3B4A3C2A41C0F6FF42C0F7FFE5
:100EF800000EF86E0800FFFFF5CF4DF04D6601D0EB
:100F080001D0DFD601D000D039C0D9FF3AC0DAFF0E
:100F1800000EDF6E00D01200FFFFFFFF1C6E000EF8
:100F2800216E1C501C6E000E226E1C50060E1902FB
:100F3800F350196E00D0780E196401D001D011D089
:100F48001C6E000E196E1C50070E1A6001D001D0DD
:100F580002D01A2A06D01C6E000E1A6E1C5001D040
:100F680000D0040E192619380F0B0F0B216E1950DB
:100F78000F0B226E1A50B00F106E87EC0BF0215039
:100F8800100F106E87EC0BF022C010F087EC0BF0FE
:100F9800ADD017C0D9FF18C0DAFFDF50236EDF0EBF
:100FA800236401D001D003D0560E235E00D01F0E5B
:100FB800236401D001D006D0B10E236401D001D042
:100FC80081D000D01C6E200E236E1C507BD07AD0AE
:100FD8001C6E000E246E1C50050E246401D001D036
:100FE80002D078D077D02450010DE00E2324106E63
:100FF800116AFF0E1122000E136E060E126E23ECFC
:101008000BF0380E10241C6EFA0E11201D6EF350D2
:101018001C241E6EF4501D201F6E1EC0F6FF1FC03C
:10102800F7FF000EF86E0800FFFFF5CF20F0D8900C
:101038002034166E93EC0BF0242A050E246401D09C
:1010480001D0D1D747D046D01C6E000E246E1C505C
:10105800050E246401D001D002D03CD03BD02450EE
:10106800010DE00E2324106E116AFF0E1122000EEE
:10107800136E060E126E23EC0BF0380E10241C6E45
:10108800FA0E11201D6EF3501C241E6EF4501D2004
:101098001F6E1EC0F6FF1FC0F7FF000EF86E080097
:1010A800FFFFF550FF0A206ED8802034166E93ECAF
:1010B8000BF0242A050E246401D001D0D0D70AD021
:1010C80009D008D01B50000AD8B482D7010AD8B476
:1010D800BBD700D0174A182A060E19267C0E1964A9
:1010E80001D001D003D00CD00BD000D017C0D9FF4D
:1010F80018C0DAFFDF50D8A401D001D04AD700D0F9
:1011080017C0D9FF18C0DAFFDF50D8A401D001D02A
:1011180012D700D01200FFFFFFFF326E000E346EB0
:10112800325031AE01D001D00DD0311E301E2F1EED
:101138002E6C000E2F2230223122326E010E346EB8
:10114800325000D02DAE01D001D00BD02D1E2C1E58
:101158002B1E2A6C000E2B222C222D22010E341A53
:1011680000D0000E356E000E366E000E376E000E83
:10117800386E31502E102F103010D8B401D001D055
:1011880036D0326E010E336E325007D0D8902E36DC
:101198002F3630363136332A00D031AE01D001D067
:1011A800F5D701D000D0D8903536363637363836B0
:1011B8002E502A5C2F502B5830502C5831502D5817
:1011C800D8A001D001D00AD02E502A5E2F502B5A19
:1011D80030502C5A31502D5A358000D0D8903132A9
:1011E80030322F322E32332EDED701D000D0345099
:1011F800D8B401D001D009D0381E371E361E356C40
:10120800000E36223722382200D035C02AF036C0E8
:101218002BF037C02CF038C02DF000D01200FFFFA3
:10122800FFFF000E256E000E266E000E276E000EC4
:10123800286E2350201021102210D8B401D001D0DC
:1012480035D0246E010E296E245007D0D890203650
:10125800213622362336292A00D023AE01D001D0E8
:10126800F5D701D000D0D89025362636273628362F
:1012780020501C5C21501D5822501E5823501F58C6
:10128800D8A001D001D00AD020501C5E21501D5A90
:1012980022501E5A23501F5A258000D0D89023323E
:1012A800223221322032292EDED700D025C01CF070
:1012B80026C01DF027C01EF028C01FF01200FFFF37
:1012C800FFFF7AEC0BF01A6EE20E106E1A5087ECE4
:1012D8000BF01A6EAE0E106E1A5087EC0BF01A6EE9
:1012E800A00E106E1A5087EC0BF01A6EC80E106E16
:1012F8001A5087EC0BF01A6EA60E106E1A5087EC77
:101308000BF01A6E240E106E1A5087EC0BF01A6E42
:10131800A20E106E1A5087EC0BF01A6E2F0E106E7C
:101328001A5087EC0BF01A6E810E106E1A5087EC6B
:101338000BF01A6E2F0E106E1A5087EC0BF01A6E07
:10134800400E106E1A5087EC0BF089EC0AF01A6EFA
:10135800AF0E106E1A5087EC0BF01200FFFFFFFF64
:101368000201020E116E0201000E106E19C012F079
:10137800136A01EC0AF010C01BF011C01CF01950E0
:10138800010D0201000EF324D96EDA6A0201020E81
:10139800DA221BC0DFFF19C01AF0010E1A2602015B
:1013A800000E1A24D96EDA6A0201020EDA221C50E3
:1013B800DF6E020E19261A6E000E1D6E1A5014D01A
:1013C80000D0ACA201D001D0FCD700D01D50010D37
:1013D8000201000EF324D96EDA6A0201020EDA2243
:1013E800DF50AD6E1D2A00D019501D5CD8A001D069
:1013F80001D0E7D700D01200FFFFFFFF1768186879
:1014080029D010C0D9FF11C0DAFFDF501818166EA6
:10141800104A112A1650010D9E0EF324F66EF76A33
:10142800FD0EF722F86A000EF8220800FFFFF550BB
:101438001718186E1650010D9E0EF324F66EF76AF3
:10144800FE0EF722F86A000EF8220800FFFFF5CF1B
:1014580017F000D01206D8A013061228D8B4132803
:10146800D8A401D001D0CDD700D0185017C014F09F
:10147800156A14C015F0146A1410106E1550116E08
:1014880000D01200FFFFFFFF31502E102F10301038
:10149800D8B401D001D02FD0326E010E336E325045
:1014A80007D0D8902E362F3630363136332A00D032
:1014B80031AE01D001D0F5D701D000D02E502A5C32
:1014C8002F502B5830502C5831502D58D8A001D0BF
:1014D80001D009D02E502A5E2F502B5A30502C5A4A
:1014E80031502D5A00D0D890313230322F322E322E
:1014F800332EE4D700D02AC02AF02BC02BF02CC002
:101508002CF02DC02DF01200FFFFFFFF176EB00E5C
:10151800196E1750B70E196401D001D002D030D01F
:101528002FD019C010F087EC0BF0176E100E106E4C
:10153800175087EC0BF0176E000E106E175087ECE3
:101548000BF0176E000E186E1750830E186401D03A
:1015580001D002D00ED00DD0176E000E166E1750A7
:1015680093EC0BF0182A830E186401D001D0F4D73D
:1015780000D0192AB70E196401D001D0D2D700D0F3
:101588001200FFFFFFFF000E186E000E196E000E0E
:101598001A6E000E1B6E00D010A001D001D009D029
:1015A800145018261550192216501A2217501B22AB
:1015B80000D0D8901436153616361736D890133210
:1015C8001232113210321350101011101210D8A408
:1015D80001D001D0E1D718C010F019C011F01AC01D
:1015E80012F01BC013F01200FFFF02EE00F011EE24
:1015F80000F0EE6AE550E150FCE1E250FAE101EE5C
:1016080000F011EE00F0EE6AE550E150FCE1E25026
:10161800FAE100EE89F0130EEE6AE806FDE14E6A83
:101628003E0EF66E170EF76E000EF86E0900F5CF37
:101638009CF00900F5CF9DF000016EEF00F0FFFF70
:10164800000E156E000E146E00D010A001D001D04F
:1016580005D0125014261350152200D0D8901236F7
:101668001336D8901132103211501010D8A401D06E
:1016780001D0EBD714C010F015C011F01200FFFF15
:10168800FFFFBE0EC06E1044E846FC0BC26EC2805F
:10169800C28200D0C2B201D001D0FCD7C290C350E0
:1016A800C4CF12F0136A12C013F0126A1210106E2F
:1016B8001350116E00D01200FFFFFFFFF00E976E5F
:1016C800AC8CAC8AAC80AB8EAB8CAB88AC84A10EF6
:1016D800AF6E800ECD6E9494CB680F0EBD6ECA842B
:1016E8009D8A9D80F28CF28E1200FFFFFFFF700E24
:1016F800966E000E956E8D9E8D808D828D848D8662
:101708008D8E1200FFFFFFFF000E956E8D9410C0A6
:1017180083FF8D928D968D868D821200FFFFFFFFCD
:10172800000E956E8D8416C083FF8D928D968D86E2
:081738008D821200FFFF840303
:10FA380000000000000000002F0000000007000781
:10FA48000000147F147F1400242A7F2A1200231335
:10FA58000864620036495522500000050300000082
:10FA6800001C224100000041221C000014083E082E
:10FA7800140008083E08080000005030000010106C
:10FA88001010100000606000000020100804020040
:10FA98003E5149453E0000427F40000042615149C5
:10FAA80046002141454B31001814127F10002745AC
:10FAB800454539003C4A49493000017109050300B0
:10FAC800364949493600064949291E00003636009C
:10FAD80000000056360000000814224100001414EB
:10FAE80014141400004122140800020151090600F0
:10FAF800324959513E007E1111117E007F49494912
:10FB080036003E41414122007F4141221C007F498D
:10FB1800494941007F09090901003E4149497A00E4
:10FB28007F0808087F0000417F4100002040413FD6
:10FB380001007F08142241007F40404040007F02BE
:10FB48000C027F007F0408107F003E4141413E00C7
:10FB58007F09090906003E4151215E007F091929E4
:10FB6800460046494949310001017F0101003F40F3
:10FB780040403F001F2040201F003F4038403F00CA
:10FB880063140814630007087008070061514945A9
:10FB98004300007F41410000552A552A5500004185
:10FBA800417F000004020102040040404040400040
:10FBB8000001020400002054545478007F48444453
:10FBC8003800384444442000384444487F003854BE
:10FBD80054541800087E090102000C5252523E008B
:10FBE8007F080404780000447D4000002040443D24
:10FBF80000007F102844000000417F4000007C0482
:10FC0800180478007C080404780038444444380018
:10FC18007C1414140800081414187C007C080404CC
:10FC28000800485454542000043F444020003C40FD
:10FC380040207C001C2040201C003C4030403C0000
:10FC48004428102844000C5050503C004464544C44
:10FC58004400083E4141000000007F0000000041D0
:10FC6800413E0800100810201000000000000000AD
:10FC780000081C3E7F0060787E786000007F3E1C94
:10FC88000800061E7E1E0600000814227F00605829
:10FC980046586000007F22140800061A621A0600FF
:10FCA8007E7E7E00000000000000000020545556B3
:10FCB800780020545655780020565556780020561E
:10FCC80055567900205554557800205454547800DE
:10FCD800205454547800384444442000385455562D
:10FCE80018003854565518003856555618003855C7
:10FCF8005455180000447D42000000467D40000035
:10FD080000467D42000000457C41000000000000E4
:10FD180000007C0A05067900384445463800384614
:10FD28004544380038464546380038464546390087
:10FD380038454445380008082A0808007864544CB7
:10FD48003C003C4041227C003C4241227C003C4239
:10FD580041207C003C4140217C000C5051523C0029
:10FD68000000000000000C5150513C000000000051
:10FD7800000000000000000000000000000000007B
:10FD8800000000000000000000000000000000006B
:10FD980000060909060000C1814001C0804101C078
:10FDA800804100C1814001C0804100C1814000C143
:10FDB800814001C0804101C0804100C1814000C133
:10FDC800814001C0804100C1814001C0804101C023
:10FDD800804100C1814001C0804100C1814000C113
:10FDE800814001C0804100C1814001C0804101C003
:10FDF800804100C1814000C1814001C0804101C0F3
:10FE0800804100C1814001C0804100C1814000C1E2
:10FE1800814001C0804101C0804100C1814000C1D2
:10FE2800814001C0804100C1814001C0804101C0C2
:10FE3800804100C1814000C1814001C0804101C0B2
:10FE4800804100C1814001C0804100C1814000C1A2
:10FE5800814001C0804100C1814001C0804101C092
:10FE6800804100C1814001C0804100C1814000C182
:10FE7800814001C0804101C0804100C1814000C172
:10FE8800814001C0804100C1814001C0804101C062
:10FE9800804100C1814000C0C101C30302C2C6063F
:10FEA80007C705C5C404CC0C0DCD0FCFCE0E0ACAAA
:10FEB800CB0BC90908C8D81819D91BDBDA1A1EDEFA
:10FEC800DF1FDD1D1CDC14D4D515D71716D6D212AA
:10FED80013D311D1D010F03031F133F3F23236F6BA
:10FEE800F737F53534F43CFCFD3DFF3F3EFEFA3A6A
:10FEF8003BFB39F9F83828E8E929EB2B2AEAEE2EFA
:10FF08002FEF2DEDEC2CE42425E527E7E62622E269
:10FF1800E323E12120E0A06061A163A3A26266A6B9
:10FF2800A767A56564A46CACAD6DAF6F6EAEAA6A29
:10FF38006BAB69A9A86878B8B979BB7B7ABABE7E79
:10FF48007FBF7DBDBC7CB47475B577B7B67672B229
:10FF5800B373B17170B050909151935352929656B9
:10FF68005797559594549C5C5D9D5F9F9E5E5A9AE9
:10FF78009B5B99595898884849894B8B8A4A4E8E79
:10FF88008F4F8D4D4C8C44848545874746868242E9
:10FF9800438341818040010000000A0000006400A2
:10FFA8000000E803000010270000A086010040427E
:10FFB8000F008096980000E1F50500CA9A3B204999
:10FFC800203D20256C64205B75415D0D0020552087
:10FFD8003D20256C64205B6D565D0D002050203D52
:10FFE80020256C64205B75575D0D002050574D200F
:08FFF8003D202564200D0000EE
:020000040030CA
:06000100220A000082014A
:060008000FC00FE00F40E5
:00000001FF
